:1000000045C0CBC15EC05DC05CC05BC05AC059C0BA
:1000100058C057C056C055C054C053C052C051C03C
:1000200050C04FC04EC00403090426037700770078
:1000300077002E0069006E0066006F006C0065009E
:10004000780069006B006F006E002E006400650090
:1000500018035500530042002D00440069006E0053
:10006000670065006E00730012011001FF000008B8
:10007000C016DC05000101020001090212000101A5
:1000800000C00A09040000000000000011241FBE87
:10009000CFE5D4E0DEBFCDBF10E0A0E6B0E0E8EFF2
:1000A000F5E002C005900D92A236B107D9F710E035
:1000B000A2E6B0E001C01D92A639B107E1F729D050
:1000C00099C29ECFFC01109262008181813069F05B
:1000D000813018F0823089F40BC0828180936200F5
:1000E00083818093630022E00CC080916A0006C087
:1000F000828180936A0020E004C081E080936200E6
:1001000021E082E690E090937B0080937A00822F3A
:1001100008958FEF81BB12BA84BB87BB2EE140E309
:1001200055E703C0CA010197F1F72150D9F78AEFCB
:1001300081BB85E083BF21D0789420E04CE251E080
:1001400008C0FA013197F1F70197D9F72F5F2A30EC
:1001500019F088EE93E0F5CF10926A0015D008B63A
:1001600000FEFCCF88B7816088BF80916A0087FD60
:1001700002C085BBF3CF88BBF1CF85B7836085BF55
:100180008BB780648BBF08951F93CF93DF939091BB
:100190007C00935097FD8DC020917900809178006C
:1001A0008D3209F084C0983009F081C0CCE0D0E0F5
:1001B000C21BD109C058DF4F83EC80936C008AE5E5
:1001C0008093600010926B009881892F807621F0D7
:1001D000CE0178DF282F62C02A81109275008981B4
:1001E000882349F49F7119F481E08093750010927F
:1001F000760022E04DC0853019F420937D0047C081
:100200008630B1F58B81813019F488E690E004C026
:10021000823041F48AE790E090937B0080937A00EB
:1002200022E122C08330F9F48A81882341F486E2F6
:1002300090E090937B0080937A0024E015C0813099
:1002400041F48AE290E090937B0080937A0026E26A
:100250000BC0823041F480E590E090937B00809366
:100260007A0028E101C020E080E480936B0016C092
:10027000883021F421E08FE790E00CC0893019F438
:1002800020937F0004C08A3011F421E001C020E0F7
:1002900085E790E090937B0080937A008F8188239C
:1002A00021F48E81821708F4282F20936100109288
:1002B0007C008091600084FF49C0809161008F3F85
:1002C00009F444C0182F893008F018E0811B80938E
:1002D000610080916C0098E8892780936C0011235D
:1002E00041F120917A0030917B0080916B0086FF74
:1002F0000DC0ADE6B0E080E090E0F901E80FF91F35
:10030000E491ED9301961817C1F708C0912FD90118
:10031000EDE6F0E08D9181939150E1F71150812F3E
:1003200090E01F5F0196820F931F90937B00809354
:100330007A008DE690E0612F2CD0612F6C5F6C30DD
:1003400019F08FEF809361006093600094E180B3B7
:10035000857031F49150D9F710927D00109277009A
:10036000DF91CF911F910895A82FB92F80E090E0E1
:1003700041E050EA609530E009C02D9182279795C1
:10038000879510F084279527305EC8F36F5FA8F338
:100390000895EADF8D939D930895CF93CFB7CF93C0
:1003A000C395809BE9F7809B09C0809B07C0809B19
:1003B00005C0809B03C0809B01C0A1C0DF93C0919A
:1003C0007900DD27C058DF4F809B02C0DF91EBCF63
:1003D0002F930F931F9300B32FEF00FB20F94F9340
:1003E0003F9310B34FEF012700FB21F93BE031C0F1
:1003F0004E7F012F10B3216028C0102F4D7F226047
:10040000000000B329C04B7F2460012F000010B30F
:100410002BC010B3477F28602AC04F7E00B32061F5
:100420002CC04F7D10B320622FC04F7B00B32064DF
:1004300032C0422700B349934FEF0000102710FB52
:1004400020F910B31570C9F1297F91F2012700FB43
:1004500021F900B3237F89F2315058F1102710FBA6
:1004600022F910B3277E79F2012700FB23F92F7CB4
:1004700081F200B3102710FB24F92F7971F200C02C
:1004800010B3012700FB25F92F7359F200C000B308
:10049000102710FB26F9223040F200C010B30127CC
:1004A00000FB27F9243028F64F77206810B30000AE
:1004B000F9CF10E41ABF002717C03B503195C31B7A
:1004C000D04010E41ABF0881033CE9F00B34D9F0A6
:1004D000209177001981110F1213EDCF093641F1E8
:1004E0000D3211F0013E39F700937E003F914F919C
:1004F0001F910F912F91DF91CAB7C6FD51CFCF91B8
:10050000CFBFCF91189520917E00222379F31091CF
:100510007C00112311F5343012F130937C002093CC
:100520007800109179003BE0311B3093790017C0BF
:1005300000917C0001308CF40AE53091600034FDBC
:1005400010C000936000CCE6D0E00FC02795A8F45F
:100550005150A9F4220F0000F9CF4AE503C042ED43
:1005600001C0432FC4E1D0E032E011B31560909A8E
:1005700011BB02B320E415E05F93012756E002BBF4
:10058000279520F4515021F4220FF9CF012756E08E
:1005900000003B5A02BBD0F2279528F4515029F4B1
:1005A000220F0000F9CF012756E0279502BB20F467
:1005B000515021F4220FF9CF012756E0299133231E
:1005C00002BB21F60A7F10917D00110FC651D04069
:1005D00002BB11F01093770010E41ABF016011B351
:1005E0001A7F402F4A7F5F9100C000C002BB11BB41
:0805F00042BB7CCFF894FFCF61
:0205F8005AFFA8
:00000001FF
